:100000000C9443010C94BC0A0C94950A0C946B015B
:100010000C946B010C94880C0C946B010C945A0C8E
:100020000C94CD0C0C946B010C946B010C946B0133
:100030000C946B010C946B010C946B010C946B0190
:100040000C944B0A0C946B010C94090B0C94E30A6E
:100050000C946B010C946B010C946B010C946B0170
:100060000C943B0B0C946B016803180172681880A8
:10007000234020034C69676874734F4E04034F4E4E
:10008000042020202020BE5004B03B805F50046834
:100090003B0205680576380A01285004683B282F82
:1000A0006805183802004F680576380A00295004A0
:1000B000683B212650046832101E50046832111F1C
:1000C000C004BF1103696804800200EE8003680168
:1000D000EA1804FF0200E16804C00200AEC0036831
:1000E00001AA6818802340200342542041756469A6
:1000F0006F04032020042020202020F36818802390
:100100004020032041555820492F5004032020044B
:100110002020202020E968188023402003555342E6
:10012000617564696F04032020042020202020A131
:1001300068188023402003432E2044697363200401
:10014000032020042020202020C368188023402082
:10015000034C6F6E677761766504032020042020CE
:10016000202020BC681880234020034D2E2057619A
:1001700076652004032020042020202020D5681844
:100180008023402003464D20626E64203204032009
:1001900020042020202020C268188023402003460D
:1001A0004D20626E64203104032020042020202092
:1001B00020C16818802340200344414220626E64BD
:1001C0003304032020042020202020AF681880233F
:1001D00040200344414220626E6432040320200424
:1001E0002020202020AE6818802340200344414274
:1001F00020626E643104032020042020202020ADE2
:100200006805183803004E68057638030020180A80
:1002100068390209003F00010177680518380100BC
:100220004C6804BF0201D000000000240027002A0F
:100230000000000000250028002B0000000008003E
:10024000020100000304070000000000000000009D
:100250000000002300260029000404040404040410
:100260000402020202020203030303030301020465
:100270000810204080010204081020010204081028
:100280002000A50D1C1311241FBECFEFD8E0DEBF48
:10029000CDBF24E0A2E7B1E001C01D92A53BB207AB
:1002A000E1F711E0A0E0B1E0EEE4F9E202C0059070
:1002B0000D92A237B107D9F711E0C2E4D1E004C032
:1002C0002197FE010E945F13C134D107C9F70E9434
:1002D000840E0C949A140C940000833081F028F45E
:1002E000813099F08230A9F008958730A9F08830E4
:1002F000C9F08430B1F4809180008F7D03C080917B
:1003000080008F7780938000089584B58F7784BDB7
:10031000089584B58F7DFBCF8091B0008F77809357
:10032000B00008958091B0008F7DF9CFCF93DF9317
:10033000282F30E0F901E55CFD4F8491F901E35984
:10034000FD4FD491F901E75AFD4FC491CC23A1F0A0
:1003500081110E946D01EC2FF0E0EE0FFF1FE15BB9
:10036000FD4FA591B491EC91ED2381E090E009F46B
:1003700080E0DF91CF91089580E090E0FACF1F9365
:10038000CF93DF93282F30E0F901E55CFD4F849196
:10039000F901E359FD4FD491F901E75AFD4FC4919A
:1003A000CC23A9F0162F81110E946D01EC2FF0E0F3
:1003B000EE0FFF1FEF5CFD4FA591B4918FB7F8943E
:1003C000EC91111108C0D095DE23DC938FBFDF9133
:1003D000CF911F910895DE2BF8CFCF93DF9390E05C
:1003E000FC01E359FD4F2491875A9D4FFC018491F4
:1003F0008823C9F090E0880F991FFC01E95DFD4F4B
:10040000A591B491FC01EF5CFD4FC591D4916111B0
:100410000DC09FB7F8948C91209582238C9388818E
:10042000282328839FBFDF91CF910895623051F434
:100430009FB7F8943C91822F809583238C93E88119
:100440002E2BEFCF8FB7F894EC912E2B2C938FBFE0
:10045000EACF3FB7F89480913A0290913B02A09185
:100460003C02B0913D0226B5A89B05C02F3F19F074
:100470000196A11DB11D3FBFBA2FA92F982F882724
:10048000BC01CD01620F711D811D911D42E0660FFF
:10049000771F881F991F4A95D1F708952FB7F894B1
:1004A0006091360270913702809138029091390242
:1004B0002FBF08950895089508950895AF92BF92AB
:1004C000CF92DF92EF92FF920F931F93CF93DF9320
:1004D0006C017B018B01040F151FEB015E01AE184F
:1004E000BF08C017D10759F06991D601ED91FC9171
:1004F0000190F081E02DC6010995892B79F7C5019E
:10050000DF91CF911F910F91FF90EF90DF90CF90EF
:10051000BF90AF900895FC01538D448D252F30E09E
:10052000842F90E0821B930B541710F0CF96089500
:1005300001970895FC01918D828D981761F0A28D2D
:10054000AE0FBF2FB11D5D968C91928D9F5F9F73F3
:10055000928F90E008958FEF9FEF0895FC01918DA9
:10056000828D981731F0828DE80FF11D858D90E016
:1005700008958FEF9FEF0895FC01918D228D892FB3
:1005800090E0805C9F4F821B91098F73992708959B
:100590008EE392E00E94BC0221E0892B09F420E066
:1005A000822F089580E090E0892B29F00E94C802F4
:1005B00081110C9400000895FC01A48DA80FB92F9F
:1005C000B11DA35ABF4F2C91848D90E001968F737B
:1005D0009927848FA689B7892C93A089B1898C919A
:1005E000837080648C93938D848D981306C00288E9
:1005F000F389E02D80818F7D80830895EF92FF92B3
:100600000F931F93CF93DF93EC0181E0888F9B8D35
:100610008C8D98131AC0E889F989808185FF15C0EF
:100620009FB7F894EE89FF896083E889F989808112
:100630008370806480839FBF81E090E0DF91CF91E1
:100640001F910F91FF90EF900895F62E0B8D10E003
:100650000F5F1F4F0F731127E02E8C8D8E110CC072
:100660000FB607FCFACFE889F989808185FFF5CFBD
:10067000CE010E94DC02F1CFEB8DEC0FFD2FF11DBE
:10068000E35AFF4FF0829FB7F8940B8FEA89FB89FA
:1006900080818062CFCFCF93DF93EC01888D882358
:1006A000B9F0AA89BB89E889F9898C9185FD03C0D5
:1006B000808186FD0DC00FB607FCF7CF8C9185FFBA
:1006C000F2CF808185FFEDCFCE010E94DC02E9CF21
:1006D000DF91CF9108952091BA01260F3327331F60
:1006E00021323105ECF420910902FC0190E080E018
:1006F000243069F082E00895A091BA012191AC0103
:1007000046565E4FA40FB52FB11D2C930196861748
:1007100098F38091BA01680F6093BA0180E0089560
:1007200081E008951092090281E0809308021092FE
:10073000E30161E082E10E94BF0161E083E10E9488
:10074000BF01E9EBF0E080818E7F808380818D7F27
:10075000808388E48093B80085E48093BC0008958A
:10076000CF93DF9391E0909399018823B9F0C091E2
:10077000B800D091BA008091BC008A7B8093BC0005
:1007800060E082E10E94BF0160E083E10E94BF015E
:100790000E949203D093BA00C093B800DF91CF912A
:1007A00008950895E091E2018091E101E81730F4A5
:1007B000F0E0E758FE4F808190E008958FEF9FEFC3
:1007C00008959091E2018091E1012FEF3FEF98179A
:1007D00048F4E92FF0E0E758FE4F208130E09F5FBA
:1007E0009093E201C90108958091E1019091E201A5
:1007F000891B990B0895CF92DF92EF92FF920F938E
:100800001F93CF93DF937C01CB018A0120910F02CC
:10081000222389F0EB016B01C40ED51ECC15DD053A
:1008200069F06991D701ED91FC910190F081E02D83
:10083000C7010995F3CF642F0E946B03C801DF91B4
:10084000CF911F910F91FF90EF90DF90CF9008957F
:10085000CF93DF931F92CDB7DEB7698320910F024C
:100860002223F9F020913202203258F021E030E0CA
:10087000FC013383228390E080E00F90DF91CF91E1
:10088000089580911002E82FF0E0EF5EFD4F99810E
:1008900090838F5F809310028093320281E090E01A
:1008A000ECCF61E0CE0101960E946B03F7CF90E0A0
:1008B00080E00895FC01848195812281338128178D
:1008C000390771F0860F971F608171810E944B1369
:1008D0000680F781E02DE80FF91F808190E00895F0
:1008E0008FEF9FEF0895FC018481958122813381F0
:1008F0002817390741F0860F971F608171810E9488
:100900004B13958384830895FC01462F2281338104
:10091000C9010196608171810E944B1364817581C8
:100920008617970781F0A681B781A20FB31F4C935A
:10093000828193810196608171810E944B13938320
:10094000828380E008958FEF0895EF92FF920F93D6
:100950001F93CF93DF937C01062F10E0B80181EA4B
:1009600094E00E948404D0E0C0E0C017D10758F49E
:10097000F701EC0FFD1F649170E081EA94E00E94A2
:1009800084042196F2CFDF91CF911F910F91FF90B8
:10099000EF900895CF93DF93FC01C281D3818481CE
:1009A0009581C817D907C9F0A681B781A80FB91FCB
:1009B0002C910196608171810E944B13C817D90751
:1009C00039F095838483822F90E0DF91CF91089551
:1009D0001582148213821282F6CF8FEF9FEFF5CF2C
:1009E000FC0160817181848195819B01281B390BF9
:1009F00082819381820F931F0E944B130895DC0123
:100A0000ED91FC910190F081E02D099480917801A5
:100A10008823B9F080917701882399F06CE08EE00B
:100A200092E00E94A50467E087E092E00E94A5049E
:100A300067E080E092E00E94A50461E08AE00C9407
:100A4000BF0160E08AE00E94BF0167E08AE192E0B6
:100A50000C94A5048F929F92AF92BF92CF92DF9297
:100A6000EF92FF924B015C010E9429026B017C0115
:100A700024E0C21AD108E108F1080E9429026C1989
:100A80007D098E099F09681579058A059B05A8F3DC
:100A9000FF90EF90DF90CF90BF90AF909F908F909E
:100AA00008958091DA03882319F060E00C94BF0167
:100AB0002D980895882349F08091DA03882319F04E
:100AC00061E00C94BF012D9A08950C945105CF93C9
:100AD000DF93EC018091DB03823019F481E00E9406
:100AE0005A05299ABE0190E080E00E942A052998C3
:100AF0008091DB03823031F40E945105DF91CF9168
:100B00000C945105DF91CF9108958F929F92AF92EF
:100B1000BF92CF92DF92EF92FF92CF934B015C0195
:100B2000219A8FEF88169806A806B806C1F4219A74
:100B300080E093E20E94670560EC78E080E090E05E
:100B40000E942A0580E392E0CF91FF90EF90DF9022
:100B5000CF90BF90AF909F908F900C94670580E0EE
:100B600093E20E94670560E871E180E090E00E94F6
:100B70002A05C0E2C12CD12CE12C90E8F92ED50138
:100B8000C4018C219D21AE21BF21892B8A2B8B2B67
:100B900089F080E392E00E94670560E976E080E0FA
:100BA00090E00E942A05F694E794D794C794C15028
:100BB00031F7C8CF80E392E00E94670560E372E0FE
:100BC00080E090E0EECFCF9329E534E0F901019089
:100BD0000020E9F79F012A553440C091540433277F
:100BE0004C2F50E0BA0161507109261B370B30932E
:100BF0004F0420934E04682F70E0675A7B4F86E1C4
:100C000091E00E948A1480911601803219F486E8DE
:100C100080931601CB5FC0931101EC2FF0E0319669
:100C200020E090E0A92FB0E0A05FBE4F4C912427B8
:100C30009F5FC917B8F7E05FFE4F208360911101F5
:100C400070E06E5F7F4F89EA94E00E948404C0E008
:100C50002C2F30E08091110190E0019682179307CC
:100C60005CF0205F3E4FF901608170E089EA94E01A
:100C70000E948404CF5FECCFCF91089585ED8093DF
:100C8000BC0080910B0290910C02A0910D02B091DA
:100C90000E020796A11DB11D23E0B695A795979565
:100CA00087952A95D1F72091BC0024FD03C01092AE
:100CB0000902089540910B0250910C0260910D02BF
:100CC00070910E02452B462B472B69F30097A10527
:100CD000B10541F02AE22A95F1F700C00197A10978
:100CE000B109E1CF80910A020C94B003FC01868126
:100CF0009781009711F00C94011408951F93CF93DE
:100D0000DF93EC01162F0E943513181739F0612F6D
:100D1000CE01DF91CF911F910C943D13DF91CF91C4
:100D20001F9108950C943513CF93DF9390E080E0EA
:100D30000E949206C82FD0E0D0930B01C0930A0105
:100D40008AE090E00E949206282F30E0309309015B
:100D5000209308012197A9F48150873090F4E82F5F
:100D6000F0E0EA54F94F6AE10C945F13BD06CD063A
:100D7000D006D306D606D906DC0686EE91E00E94A0
:100D8000A5048AE090E00E94920690E09093090109
:100D900080930801DF91CF9108958CEC91E0EFCF23
:100DA00082EB91E0ECCF88E991E0E9CF8EE791E02A
:100DB000E6CF84E691E0E3CF8AE491E0E0CF90E0F3
:100DC00080E00E949206282F30E0309307012093A4
:100DD00006018330D9F028F4813049F0823069F07F
:100DE0000895853029F1D0F0873039F108951092B7
:100DF00077010E9406050C949406109277010E94D8
:100E000006056AE180E391E00C94A5041092770155
:100E10000E9406056AE186E191E0F6CF6AE18CEF77
:100E200090E00E94A50481E0809377010C94060570
:100E30006AE182EE90E00E94A50410927701F6CF5D
:100E40008F929F92AF92BF92CF92DF92EF92FF92DA
:100E50000F931F93CF93DF93CDB7DEB768970FB68D
:100E6000F894DEBF0FBECDBF7C01FC010081C280C3
:100E7000D38016810E944E0280907201909073017F
:100E8000A0907401B09075019B01AC01281939093B
:100E90004A095B0949015A0130E1831637E293069A
:100EA000A104B10468F060937201709373018093A0
:100EB00074019093750165E088E690E00E94A504B6
:100EC00045E050E06DED70E0C7010E942813892BCA
:100ED00029F466E087ED90E00E94A50446E050E02A
:100EE00061ED70E0C7010E942813892B19F481E09D
:100EF000809378018091340281110AC066E081E21A
:100F000092E00E94A5040E94DF0681E080933402F3
:100F100045E050E06CEC70E0C7010E942813892B7B
:100F200029F466E086EC90E00E94A50445E050E0DC
:100F300060EC70E0C7010E942813892B11F40E9415
:100F4000DF06003809F073C24FEBC41273C258E1D8
:100F5000D51270C261E081E10E94BF0180917601EB
:100F6000811105C00E94DF0681E0809376016896BA
:100F70000FB6F894DEBF0FBECDBFDF91CF911F91AA
:100F80000F91FF90EF90DF90CF90BF90AF909F9028
:100F90008F900895153009F487C0163041F766E048
:100FA0008AE990E00E94A50480917701882309F4E2
:100FB000B4C080917801882309F4AFC067E083E969
:100FC00090E08CC0193009F4E1C008F4ABC01A30CD
:100FD00009F48EC165E77AE88EE491E61B3009F4E6
:100FE00046C2C5CF183209F406C248F5133209F4D7
:100FF000CAC190F41E3009F0BACF61E08AE00E94C5
:10100000BF018CE00E949601892B09F4B4C160E015
:101010008CE00E94BF01A3C0163209F4DFC1173271
:1010200009F0A5CF80917701882321F08091780184
:10103000811156C06FE070EF8EE491E618C21C3249
:1010400009F4A6C158F4193209F4ECC16FE570EA4D
:101050008EE491E61B3209F40AC289CF1D3209F4ED
:101060009CC11E3409F083CF60E08AE068960FB619
:10107000F894DEBF0FBECDBFDF91CF911F910F91CE
:10108000FF90EF90DF90CF90BF90AF909F908F90A8
:101090000C94BF0166E08AEB90E00E94A50467ED26
:1010A00078E28EE491E6E3C166E084EB90E00E9492
:1010B000A50467E578EA8EE491E6D9C166E08EEA98
:1010C00090E00E94A5048091770167E08823E1F019
:1010D000809178018823C1F087EA90E00E94A504FE
:1010E00068960FB6F894DEBF0FBECDBFDF91CF91EB
:1010F0001F910F91FF90EF90DF90CF90BF90AF9036
:101100009F908F900C94060580EA90E00E94A504C1
:1011100067EB78E48EE491E6AAC167E378EC8EE4AD
:1011200091E6A5C166E08DE890E00E94A5046FEA13
:1011300070E58EE491E60E9485058091060190910C
:101140000701019686309105F4F49093070180938E
:1011500006016091060190E080E00E947E0668969C
:101160000FB6F894DEBF0FBECDBFDF91CF911F91B8
:101170000F91FF90EF90DF90CF90BF90AF909F9036
:101180008F900C94DF0681E090E0DFCF90E080E06C
:101190000E949206E82EF12CF0920B01E0920A01D7
:1011A00081E0E816F10409F067C06FE470EB8EE4AB
:1011B00091E60E94850587E090E090930501809379
:1011C00004018091020190910301019688309105FC
:1011D00034F59093030180930201609102018BE04A
:1011E00090E00E947E068BE090E00E949206282FFD
:1011F00030E030930301209302018150873008F0E2
:10120000B6CEE82FF0E0E85FF64F6AE10C945F138A
:1012100014092A092D093009330936093909F092D0
:101220000301E0920201D9CF86EE91E068960FB6F5
:10123000F894DEBF0FBECDBFDF91CF911F910F910C
:10124000FF90EF90DF90CF90BF90AF909F908F90E6
:101250000C94A5048CEC91E0E9CF82EB91E0E6CF11
:1012600088E991E0E3CF8EE791E0E0CF84E691E07A
:10127000DDCF8AE491E0DACF90E080E00E94920630
:1012800090E090930B0180930A01029709F06FCED2
:101290008091080190910901019690930901809332
:1012A000080120910401309105012817390734F411
:1012B00081E090E09093090180930801609108011A
:1012C0008AE090E00E947E0668960FB6F894DEBF32
:1012D0000FBECDBFDF91CF911F910F91FF90EF9087
:1012E000DF90CF90BF90AF909F908F900C9494061A
:1012F000809100019091010101968630910564F57D
:1013000090930101809300016091000188E290E0D8
:101310000E947E0688E290E00E94920690E0909300
:1013200001018093000128E1E6E3F1E0DE0111967E
:1013300001900D922A95E1F7880F991F880F991F48
:10134000E1E0F0E0EC0FFD1F8E0F9F1FFC016081BC
:101350007181828193818BC01092010110920001F2
:10136000D3CF66E087E890E00E94A50465E97AE6BD
:101370008EE491E67CC061E08CE00E94BF016AE1EE
:101380008DE690E053CF6FE170EE8EE491E66FC092
:1013900065EC7AE38EE491E66AC061E090E080E07B
:1013A0000E947E0661E08AE090E00E947E0661E095
:1013B0008BE090E00E947E0660E08EE190E00E946B
:1013C0007E0660E088E290E00E947E0660E08CE8A5
:1013D00090E00E947E060E94DF0676CF8091770122
:1013E000882321F08091780181117ACE6FE870E72F
:1013F0008EE491E63CC062E090E080E068960FB633
:10140000F894DEBF0FBECDBFDF91CF911F910F913A
:10141000FF90EF90DF90CF90BF90AF909F908F9014
:101420000C947E066FE470EB8EE491E620C0003CE5
:1014300009F09DCDF1E3DF129ACD61E085E00E94D5
:10144000BF011C3009F48DCF08F0CCCD173009F462
:1014500035CE08F0B7CD143009F41CCE08F09ACD83
:1014600067E978E68EE491E6133009F080CD68965E
:101470000FB6F894DEBF0FBECDBFDF91CF911F91A5
:101480000F91FF90EF90DF90CF90BF90AF909F9023
:101490008F900C9485051F920F920FB60F92112416
:1014A0002F933F938F939F93AF93BF938091360277
:1014B00090913702A0913802B091390230913502F3
:1014C00023E0230F2D3758F50196A11DB11D209360
:1014D00035028093360290933702A0933802B0937E
:1014E000390280913A0290913B02A0913C02B09166
:1014F0003D020196A11DB11D80933A0290933B02DB
:10150000A0933C02B0933D02BF91AF919F918F9108
:101510003F912F910F900FBE0F901F90189526E8C6
:10152000230F0296A11DB11DD2CF1F920F920FB6AD
:101530000F9211242F933F934F935F936F937F9359
:101540008F939F93AF93BF93EF93FF93E0910E011F
:10155000F0910F010995FF91EF91BF91AF919F918C
:101560008F917F916F915F914F913F912F910F904C
:101570000FBE0F901F9018951F920F920FB60F92EB
:1015800011242F933F934F935F936F937F938F9388
:101590009F93AF93BF93EF93FF93E0910C01F09172
:1015A0000D010995FF91EF91BF91AF919F918F919F
:1015B0007F916F915F914F913F912F910F900FBE4F
:1015C0000F901F9018951F920F920FB60F92112433
:1015D0002F933F934F935F936F937F938F939F933B
:1015E000AF93BF93EF93FF938EE392E00E94DC02F0
:1015F000FF91EF91BF91AF919F918F917F916F91EB
:101600005F914F913F912F910F900FBE0F901F90C0
:1016100018951F920F920FB60F9211242F938F934C
:101620009F93EF93FF93E0914E02F0914F028081E0
:10163000E0915402F091550282FD1BC0908180918F
:1016400057028F5F8F7320915802821741F0E0910B
:101650005702F0E0E25CFD4F958F80935702FF91B7
:10166000EF919F918F912F910F900FBE0F901F9030
:1016700018958081F4CF1F920F920FB60F9211240C
:101680002F933F934F935F936F937F938F939F938A
:10169000AF93BF93EF93FF938091B900887F80361B
:1016A00009F44AC0F0F5883209F4A7C018F5803172
:1016B00009F49BC0B8F4882309F4F9C0883009F410
:1016C00094C0FF91EF91BF91AF919F918F917F91C6
:1016D0006F915F914F913F912F910F900FBE0F909F
:1016E0001F901895883109F488C0803251F7809393
:1016F000070214C0803409F49DC040F48033B9F36C
:101700008833F9F68093070285ECB0C0803509F480
:1017100085C0883509F496C0883499F60E943E0643
:10172000D0CF883909F48CC038F5883729F050F4C7
:10173000883611F0803729F683E0809309021092F1
:10174000DC0157C0883809F47BC0803919F0803833
:1017500009F0B7CF8091DC01803208F071C0E091D0
:10176000DC0181E08E0F8093DC018091BB00F0E012
:10177000E454FE4F80833DC0803B39F0E0F4803A72
:1017800009F479C0883A09F09CCF84E0809309027B
:101790001092BB011092BA01E091DF01F091E001DB
:1017A00009958091BA0181110FC081E08093BA013F
:1017B00010929A0109C0803C09F4A6CF883C09F434
:1017C000A3CF883B09F07DCFE091BB0181E08E0F74
:1017D0008093BB01F0E0E656FE4F80818093BB0012
:1017E0009091BB018091BA0129C08091E40180935E
:1017F000BB0085EC8093BC0064CF90910602809181
:101800000502981758F5E091060281E08E0F80934B
:101810000602F0E0EB51FE4F8081E9CFE091060235
:1018200081E08E0F809306028091BB00F0E0EB51C7
:10183000FE4F808390910602809105029817C8F2AE
:1018400085E8D8CFE091060281E08E0F80930602F2
:101850008091BB00F0E0EB51FE4F80838091080245
:1018600081115CCF81E08093E30184EA8093BC0026
:101870001092090226CF85EC8093BC0010920902D9
:101880008091DC01803230F4E091DC01F0E0E4543E
:10189000FE4F10826091DC0170E0E091DD01F0917B
:1018A000DE018CEB91E009951092DC010ACF1092D9
:1018B000070234CF1F920F920FB60F9211242F936D
:1018C0003F934F935F936F937F938F939F93AF93C8
:1018D000BF93EF93FF9381E08093330260E08DE04C
:1018E0000E94BF01E1EBF0E08081887F8083FF915F
:1018F000EF91BF91AF919F918F917F916F915F9188
:101900004F913F912F910F900FBE0F901F90189500
:101910001F920F920FB60F9211242F933F934F9364
:101920005F936F937F938F939F93AF93BF93EF9347
:10193000FF9380E00E9496010197D9F481E00E9414
:1019400096010197B1F48091B10087608093B10056
:10195000FF91EF91BF91AF919F918F917F916F9187
:101960005F914F913F912F910F900FBE0F901F905D
:10197000189580E00E949601892B51F781E00E9422
:101980009601019729F71092330261E08DE00E94E1
:10199000BF018091B100887FD9CF1F920F920FB6FF
:1019A0000F9211242F933F934F935F936F937F93E5
:1019B0008F939F93AF93BF93CF93EF93FF93E09158
:1019C000F102F091F202C0818091F302C82380916C
:1019D000F4029091F502019649F08091F402909101
:1019E000F50201969093F5028093F4028091EF0244
:1019F00081111DC0C1116EC08091F4029091F50259
:101A0000813A910578F01092F8028091F402909159
:101A1000F5029093FB028093FA0281E08093F90231
:101A20008093EF021092F5021092F40253C080915D
:101A3000EF028130A9F4CC2309F44CC0E091F90203
:101A40008E0F8093F9028091F4029091F502F0E0FC
:101A5000EE0FFF1FE151FD4F9487838782E0E0CFB7
:101A60008091EF02823009F04FC0C11122C0E09195
:101A7000F90281E0E03768F08093F80283E0809318
:101A8000EF02E091F602F091F702309759F20995D2
:101A9000C9CF8E0F8093F9028091F4029091F502E4
:101AA000F0E0EE0FFF1FE151FD4F9487838781E047
:101AB000B7CF8091F4029091F502813A910550F0F0
:101AC00083E08093EF02E091F602F091F702309705
:101AD00009F009958091DB03813021F4C11180E088
:101AE0000E945A05FF91EF91CF91BF91AF919F91C5
:101AF0008F917F916F915F914F913F912F910F90B7
:101B00000FBE0F901F9018958091EF02833011F750
:101B1000C111E0CF87CF0F931F93CF93DF93EC01D9
:101B20008B01798368831D821C821B821A82CB0100
:101B30000E9465139F838E83A80170E060E0DF91AF
:101B4000CF911F910F910C949314CF93DF93EEE3F9
:101B5000F2E01382128288EE93E0A0E0B0E084838A
:101B60009583A683B78322E531E03183208325EC7A
:101B700030E03587248724EC30E03787268720EC57
:101B800030E0318B208B21EC30E0338B228B22EC48
:101B900030E0358B248B26EC30E0378B268B118E92
:101BA000128E138E148EEBEDF2E013821282848378
:101BB0009583A683B78384E691E0918380830E9416
:101BC0004E026093EB027093EC028093ED029093CF
:101BD000EE020E944E026093E7027093E802809347
:101BE000E9029093EA0260E870E089E994E00E94DB
:101BF0008B0D60E470E081EA94E00E948B0D60E45C
:101C000070E089EA94E00E948B0DEFEEF2E0F09331
:101C10000304E0930204118281E0848389E290E06E
:101C20009383828350981092DA03CFE0D4E01CAA09
:101C30000E944E026093EB027093EC028093ED02DF
:101C40009093EE020E944E026093E7027093E802C6
:101C50008093E9029093EA0219861A861B861886F9
:101C60001F821E821D8262E080E00E94ED0161E021
:101C700084E00E94ED0161E084E00E94BF01E0EB9E
:101C8000F0E010821092B1008DE98093B300808162
:101C900082608083E0E7F0E0808182608083E8E614
:101CA000F0E0808184608083EDE6F0E080818160F7
:101CB000808319821A8280ED97E09AAF89AF88EE0F
:101CC00093E09CAF8BAF88EC90E09EAF8DAF82E04D
:101CD0008093550410924F0410924E048BE0809331
:101CE00054041092560410925704109258040E9403
:101CF0004E02609350047093510480935204909369
:101D00005304DF91CF910895789484B5826084BDA7
:101D100084B5816084BD85B5826085BD85B58160EF
:101D200085BD80916E00816080936E00109281006D
:101D30008091810082608093810080918100816028
:101D400080938100809180008160809380008091E9
:101D5000B10084608093B1008091B0008160809375
:101D6000B00080917A00846080937A0080917A003C
:101D7000826080937A0080917A00816080937A00FB
:101D800080917A00806880937A001092C10061E0AF
:101D900085E00E94ED0161E086E00E94ED0160E0D7
:101DA0008AE00E94ED0161E08BE00E94ED0161E0BC
:101DB0008CE00E94ED0162E084E10E94ED0161E0AF
:101DC0008DE00E94ED01E0914E02F0914F0282E021
:101DD0008083E0914A02F0914B021082E0914C0224
:101DE000F0914D0280E1808310925602E091520200
:101DF000F091530286E08083E0915002F09151020D
:101E0000808180618083E0915002F0915102808155
:101E100088608083E0915002F09151028081806857
:101E20008083E0915002F091510280818F7D808308
:101E300061E085E00E94BF011092E2011092E10191
:101E400010921002109232020E9492038BE592E0EF
:101E50009093E0018093DF018CE592E09093DE01A6
:101E60008093DD0181E080930F028FE28093310245
:101E70006FE78BED92E00E942804C0913202C132DC
:101E800008F091C00E9429026B017C018091090237
:101E9000811164C082E08093090281E0809308028E
:101EA0008FEF8093070210920602C0930502A1E112
:101EB000B2E0E5EEF1E080E0C81323C11092E40146
:101EC0008091E4018E658093E4018091E30181308B
:101ED00009F01BC11092E3010E9429026B017C01F1
:101EE0008091E4018093BB0080910B0290910C02E1
:101EF000A0910D02B0910E02892B8A2B8B2B99F0A9
:101F00000E94290200910B0210910C0220910D02F7
:101F100030910E026C197D098E099F09061717076B
:101F200028073907E0F18091BC0083FDD9CF85EC0B
:101F30008093BC000E9429026B017C018091090200
:101F4000823009F4E4C0809107028F3F61F18091F3
:101F50000702803241F18091070225C080910B0277
:101F600090910C02A0910D02B0910E02892B8A2B48
:101F70008B2B09F48BCF0E94290200910B02109148
:101F80000C0220910D0230910E026C197D098E0910
:101F90009F09061717072807390708F077CF8091A0
:101FA0000A020E94B00310921002109232021092A4
:101FB0000F028EE392E09093130480931204E09159
:101FC0004E02F0914F0292E09083E0914A02F0912C
:101FD0004B021082E0914C02F0914D028FEC808315
:101FE00010925602E0915202F091530286E28083F1
:101FF000E0915002F0915102808180618083E091F4
:102000005002F0915102808188608083E0915002FB
:10201000F0915102808180688083E0915002F091BC
:10202000510280818F7D80832CED35E0309349040F
:102030002093480428EE33E030934B0420934A0465
:1020400028EC30E030934D0420934C0490935504D9
:1020500080E297E0909347048093460461E08DE02E
:102060000E94ED0192E0292E312CEE24E394F12C14
:1020700034E0C32ED12C8091340281112FC00E94F4
:1020800029024B015C0188EE482E83E0582E612C1A
:10209000712C0E942902681979098A099B09683EF6
:1020A000734081059105A8F321E0421A51086108A7
:1020B000710888EE880E83E0981EA11CB11C4114A3
:1020C00051046104710429F766E081E292E00E9404
:1020D000A5040E94DF06B1E0B0933402E09114043D
:1020E000F0911504E830F105B0F5E758FF4E0C9477
:1020F0005F13A91064117A119D11C611DB11EF1144
:1021000010129D9191938F5FD7CE85EE11CF809164
:102110000B0290910C02A0910D02B0910E02892B3E
:102120008A2B8B2B09F40ACF0E94290200910B0203
:1021300010910C0220910D0230910E026C197D0954
:102140008E099F09061717072807390708F0F6CEEA
:1021500026CF10925604809133028823E1F089EA59
:1021600094E00E94F00418161906ACF489EA94E091
:102170000E94CA04EC0180E00E949601019731F4AC
:10218000B12CA12CC331D10508F470C1BE0189EA7C
:1021900094E00E9473048091120490911304DC0176
:1021A000ED91FC910084F185E02D0995892B81F05A
:1021B0008091120490911304DC01ED91FC91028452
:1021C000F385E02D0995BC0189E994E00E9484041F
:1021D00080911604909117048230910509F49BC1F7
:1021E00008F058C1009709F463C1019709F475C15B
:1021F000809133028823C9F181EA94E00E94F004BF
:102200001816190694F50E944E020091E7021091EB
:10221000E8022091E9023091EA02601B710B820B07
:10222000930B6A30710581059105F8F081EA94E01D
:102230000E94CA04EC0180E00E949601019731F4EB
:10224000B12CA12CC132D1050CF4E2C1BE0181EA4E
:1022500094E00E9473040E944E026093E702709320
:10226000E8028093E9029093EA02809110048823A7
:1022700071F00E944E0260E084E00E94BF0170E0B5
:1022800060E080911204909113040E94FF040E9468
:102290004E0261347F418105910548F08BE00E9438
:1022A0009601019721F460E08BE00E94BF0180E07D
:1022B00090E0892B09F4DFCE0E94C802882309F43C
:1022C000DACE0E940000D7CE109258041092570424
:1022D00080E00E94E30530921504209214040E94CD
:1022E0004E02609350047093510480935204909373
:1022F000530431CF0E944E020091500410915104BA
:102300002091520430915304AB01BC01401B510B8E
:10231000620B730B8091480490914904B0E0A0E0F7
:10232000481759076A077B0708F415CF83E090E048
:1023300090931504809314040ECF8091570420913C
:102340004E0430914F048217130680F48F5F809300
:1023500057048091580491E0980F909358040E947C
:10236000E305D0921504C0921404B9CFA5E0B0E003
:10237000B0931504A09314041092580410925704BB
:10238000809156048F5F80935604E5CE0E944E02E2
:102390000091500410915104209152043091530443
:1023A000AB01BC01401B510B620B730B80914C04C1
:1023B00090914D04B3CF9091560480915504981795
:1023C00038F486E090E0909315048093140487CF4E
:1023D000A7E0B0E0B0931504A093140480CF0E944E
:1023E0004E020091500410915104209152043091FA
:1023F0005304AB01BC01401B510B620B730B80916A
:102400004A0490914B04B0E0A0E0481759076A07CE
:102410007B0708F4A0CEF0921504E09214049BCE42
:102420000E944E02009150041091510420915204D8
:1024300030915304AB01BC01401B510B620B730B79
:1024400080914A0490914B04B0E0A0E048175907EE
:102450006A077B0708F47FCE1092580480E00E9440
:10246000E305109215041092140475CE0091120425
:1024700010911304CA15DB0509F48DCE89EA94E0A6
:102480000E94CA04BC01C8010E94FF04BFEFAB1A3E
:10249000BB0AECCF8330910509F477C061E070E0AE
:1024A000049709F0A5CE89E994E00E947304ABC0BB
:1024B00089E994E00E94F004181619060CF098CEF1
:1024C00070E060E089E994E00E945A048093180467
:1024D000F0921704E09216048BCE89E994E00E94F2
:1024E000F00402970CF484CE61E070E089E994E096
:1024F0000E945A04809319048350823228F4309247
:1025000017042092160474CE61E070E089E994E02B
:102510000E9473046DCE0091190410E05801BFEFC2
:10252000AB1ABB0A89E994E00E94F004A816B90628
:102530000CF05ECE712CD0E0C0E0BE0189E994E0E1
:102540000E945A04782621960C171D07B4F7B5018E
:1025500089E994E00E945A047816190689F40E94C9
:102560004E026093EB027093EC028093ED02909325
:10257000EE0283E090E0909317048093160438CE27
:10258000D0921704C092160433CE80911804982F6D
:102590009F77903521F0982F9F7B903899F4CFE06A
:1025A000D4E09E012F50344021968091190490E090
:1025B000019682179307ECF089E994E00E94CA041F
:1025C0008B87EFCF893759F3982F9D7F983639F352
:1025D0008F3329F3883119F3982F9F7D983CF9F2B6
:1025E0006091190470E06E5F7F4F803B09F05BCF14
:1025F000D6CF91E090934304E0914604F0914704D4
:102600008BE194E009951092170410921604F0CD16
:10261000AC16BD060CF01FCE0091120410911304ED
:1026200081EA94E00E94CA04BC01C8010E94FF0430
:10263000AFEFAA1ABA0AECCF89EA94E00E947606B4
:1026400081EA94E00E94760689E994E00C9476068B
:10265000FB01DC0104C08D910590801921F44150EB
:102660005040C8F7881B990B0895F999FECF92BD89
:1026700081BDF89A992780B50895262FF999FECF44
:102680001FBA92BD81BD20BD0FB6F894FA9AF99A8F
:102690000FBE01960895AA1BBB1B51E107C0AA1FDC
:1026A000BB1FA617B70710F0A61BB70B881F991FF3
:1026B0005A95A9F780959095BC01CD010895EE0F2C
:1026C000FF1F0590F491E02D09940F931F93CF9372
:1026D000DF938230910510F482E090E0E091B30442
:1026E000F091B40430E020E0B0E0A0E0309799F43D
:1026F0002115310509F44AC0281B390B2430310556
:10270000D8F58A819B816115710589F1FB0193835D
:102710008283FE0111C040815181028113814817DB
:102720005907E0F04817590799F4109761F012968D
:102730000C93129713961C933296CF01DF91CF9191
:102740001F910F9108950093B3041093B404F4CF34
:102750002115310551F04217530738F0A901DB016B
:102760009A01BD01DF01F801C1CFEF01F9CF9093CC
:10277000B4048093B304CDCFFE01E20FF31F819325
:1027800091932250310939832883D7CF2091B10406
:102790003091B204232B41F4209132013091330166
:1027A0003093B2042093B104209130013091310173
:1027B0002115310541F42DB73EB7409134015091B8
:1027C0003501241B350BE091B104F091B204E217FE
:1027D000F307A0F42E1B3F0B2817390778F0AC0144
:1027E0004E5F5F4F2417350748F04E0F5F1F509321
:1027F000B2044093B104819391939FCFF0E0E0E065
:102800009CCFCF93DF930097E9F0FC0132971382BE
:102810001282A091B304B091B404ED0130E020E045
:102820001097A1F420813181820F931F2091B10470
:102830003091B2042817390709F061C0F093B2044F
:10284000E093B104DF91CF910895EA01CE17DF073D
:10285000E8F54A815B819E0141155105B1F7E90117
:10286000FB83EA8349915991C40FD51FEC17FD07EB
:1028700061F4808191810296840F951FE90199830B
:102880008883828193819B838A83F0E0E0E01296C3
:102890008D919C9113970097B9F52D913C911197CB
:1028A000CD010296820F931F2091B1043091B204A2
:1028B0002817390739F6309751F51092B404109261
:1028C000B304B093B204A093B104BCCFD383C2834A
:1028D00040815181840F951FC817D90761F44E5F5D
:1028E0005F4F88819981480F591F518340838A81A6
:1028F0009B81938382832115310509F0B0CFF0933A
:10290000B404E093B3049ECFFD01DC01C0CF138279
:102910001282D7CFFB01DC0102C001900D92415021
:102920005040D8F70895DC0101C06D9341505040EC
:10293000E0F7089511E0C2E4D1E004C0FE010E9476
:0E2940005F132196C334D107C9F7F894FFCF77
:10294E000100010001000100010001005D025D02B5
:10295E00C80080234232000000000000000000008A
:10296E000000000000000000000000000000000059
:10297E000000B50480007D824E61BD424E613DC2B5
:10298E004E61DD224E615DA24E619D624E61000080
:10299E000000FE025E028B024B03BC029A02AE02E4
:1029AE00000000002804FB035704D103F403E103E5
:0229BE00D20342
:00000001FF
